:020000040000FA
:0600000093EF26F0120050
:0600080004EF08F01200F5
:060018000CEF08F01200DD
:0610000093EF26F0120040
:021006001200D6
:0610080085EF0AF0120062
:06101800ADEF0AF012002A
:02101E000100CF
:0C1020005E4D0000600000005800000061
:04102C0092808050DE
:10103000010B1200EEEC19F0ECEC1BF00BE0FD0ED6
:10104000DB06FE0E01E2DB06500EE66EA1EC26F09A
:10105000E552F2D70DEF1AF048EC1CF0E00E4DEC23
:101060001BF092908080280E73EC1CF0DF6EA80EAF
:101070004DEC1BF0F28EDF50E5520DEF1AF048EC0C
:101080001CF0020E73EC1CF0050E73EC1CF0DF6E0E
:10109000F28EDF50E5520DEF1AF0EEEC19F0F29EF1
:1010A00092908090020E1FEC1AF0FE0EDB5002E0D0
:1010B00092908080640E1FEC1AF092908080F28EE5
:1010C0000DEF1AF0CFEC1BF0010EDB6ADF6A080EA1
:1010D000DF5C1AE2D4DF000912E0010EDF5206E005
:1010E000DFCFF3FFE846FE0BF306FCE1146E010EC2
:1010F000DBCFE7FF1450E712010EE7CFDBFF780EDE
:101100001FEC1AF0DF2AE3D7010EDB50146E020E3B
:10111000E15C02E2E16AE552E16E14500DEF1AF073
:10112000CFEC1BF0DF6A080EDF5C1BE2FE0EDB502B
:10113000DF5206E0DFCFF3FFE8327F0BF306FCE17E
:10114000E76E010EE7CFDBFFDB92DB94DB96DB98EB
:10115000DB9ADB9CDB9EDBCFE6FF9FDFE552DF2ADD
:10116000E2D7690E1FEC1AF0020EE15C02E2E16ABE
:10117000E552E16E0DEF1AF0EEEC19F0E652FE0EBC
:10118000DB50550812E1550ECDEC1AF0DF6A080E5F
:10119000DF5C0EE2DF50EA6AF40FE96E000EEA222D
:1011A000EF50CDEC1AF0DF2AF2D7CC0ECDEC1AF0CE
:1011B000E5520DEF1AF0EEEC19F0080EE126010EE3
:1011C000F36E020EF3CFDBFF010EF36E030EF3CFCF
:1011D000DBFF040EDB6A070EDB6A010EDB6A080E1A
:1011E000F36E010E48EC1BF006E2BDEC1AF0EF6A5C
:1011F000010EDB2AF4D730DFE76E060EE7CFDBFF08
:10120000DB5003E10001FC5104E00001FD6B000E26
:101210008CD0F00ECDEC1AF0010EDB6ADF6A2FDF06
:10122000000902E0020EDF6E780E1FEC1AF027DFD5
:10123000000902E0000EDF80780E1FEC1AF0030EAA
:10124000DF5C59E0DF50000805E2DF407F0BE76E0E
:10125000050E24D00001FD51F36E030E48EC1BF087
:101260000CE2020EDBCFE6FFBDEC1AF0EF50E552C8
:10127000E714000806E2010E07D0030EDB50FD5D07
:1012800002E0000E01D0010EE76E050EE7CFDBFF96
:10129000DB5006E1030EDB50E76E040EE7CFDBFF09
:1012A000050EDB5006E0BDEC1AF0020EDB50EF122B
:1012B00007D0020EDB1C146EBDEC1AF01450EF16B2
:1012C000050EDBCFE6FFE9DEE552030EDB2A020E58
:1012D000DB50020D020EF3CFDBFFDB5006E1010E07
:1012E000DB2AF36E020EF3CFDBFF080EF36E010E66
:1012F00048EC1BF093E3410EF36E030E48EC1BF039
:1013000003E20001FD6B0FD0040EDBCFFDF0000106
:10131000FD5102E0000E01D0010EFC6F010EF36ED4
:10132000070EF3CFDBFF070EDB50146E080EE15CF7
:1013300002E2E16AE552E16E14500DEF1AF000018D
:10134000FD6BFC6BDBEF08F0EEEC19F0C5EC1AF06E
:101350004E0ECDEC1AF0FE0EDBCFE6FFE1DEE552DD
:10136000FD0EDBCFE6FFDCDEE5520A0E1FEC1AF0C5
:10137000C5EC1AF0480ECDEC1AF00A0EE66EE66ADD
:1013800059DEE552E5520DEF1AF0EEEC19F00E0EB3
:10139000E126C5EC1AF0BE0ECDEC1AF0DF6A090E9C
:1013A000DF5C13E28FDEE66ED950050F146EDACFE4
:1013B00015F0DF500F011424E96E000EDA20EA6EFA
:1013C000E552E750EF6EDF2AEAD7C5EC1AF09290AB
:1013D0008080440ECDEC1AF0050EDB50FF0808E1CA
:1013E0000C0EDB50100804E0F36A800EF46E85D01A
:1013F000010EDB6A020EDB6A060EDBCF14F020EC76
:101400001BF0050EDB50146E156AD2EC1AF0145066
:10141000EE121550ED12100E0001F45D56E1D2EC03
:101420001AF0010E0F0B06E0EC52D890ED32EF32BD
:10143000E806FAE1010EDBCF14F0020EDBCF15F067
:1014400020EC1BF0D2EC1AF0400EEE5E000EED5ACE
:101450000C0EDBCFE6FF0B0EDB50E552E75CE66ED1
:10146000D950030F02EC1CF0E552E750EE6EED6A26
:1014700074EC1BF014C015F0146A6DEC1BF00C0E2C
:10148000DB5012E00C0EDB50146E156A030EDBCF3E
:1014900008F0040EDBCF09F014C00DF015C00EF0FB
:1014A0006DEC26F07BEC1BF0010EDBCF16F0020E8C
:1014B000DBCF17F0030EDB501624146E040EDB5046
:1014C0001720156E6DEC1BF012D0010EDBCF08F06B
:1014D000020EDBCF09F07BEC1BF0D950030F02ECBE
:1014E0001CF0040ED890EE36ED36E806FBE174EC05
:1014F0001BF014C0F3FF15C0F4FF0E0EE15C02E216
:10150000E16AE552E16E0DEF1AF06AEC1AF000EEB6
:1015100000F0140EE80403E3EECFE4FFFBD700EE87
:1015200014F0080EE80403E3EECFE4FFFBD7E65225
:10153000CED8E55200EE1BF0080EE80403E3E5CF39
:10154000EDFFFBD700EE13F0140EE80403E3E5CF44
:10155000EDFFFBD796EC1AF01100D8CFE4FFE0CFF7
:10156000E4FFE46E6AEC1AF000EE00F0140EE804FA
:1015700003E3EECFE4FFFBD700EE14F0080EE8041F
:1015800003E3EECFE4FFFBD7E65228D9E55200EEA5
:101590001BF0080EE80403E3E5CFEDFFFBD700EEF8
:1015A00013F0140EE80403E3E5CFEDFFFBD796EC50
:1015B0001AF0E550E5CFE0FFE5CFD8FF1000CFEC03
:1015C0001BF03FDAA2EC21F0200E0001B85D02E032
:1015D000A2EC21F0AAEC1BF005E0B8EC11F0000140
:1015E000F26BF36B00019C519D1168E090519111D9
:1015F00018E1A86BA96B060EA7AF02D0D89003D054
:10160000A65D000EA75904E2A62B000EA72309D061
:10161000A66BA76B94DE000904E0010E0001906F39
:10162000916B00019051911142E0AFDEF3CFDEFFEC
:10163000F4CFDDFF91EC1AF0153404E314500008E8
:10164000C90E15541AE2DECF16F0DDCF17F0D89090
:10165000175004E6000E165C7D0E17580EE20001CE
:10166000A86BA96B9251931105E0DECF94F0DDCF0A
:1016700095F01DD09269936B1AD00001A82B000E33
:10168000A923A93514E2A8510408000EA9550FE2B8
:10169000946B800E956F906B916B926B936B030EB6
:1016A0009E1905E19F5103E1020E9E6F9F6B9C6B9B
:1016B0009D6B9E519F1102E069EC12F081EC13F0DA
:1016C0000001B25101E180D79DEC18F07DD70001F7
:1016D000B551B61102E1000E04D082EC1BF001E01E
:1016E000010E000901E078D0200E0001B85D74E120
:1016F00004013051730A6EE0010A69E0020A64E0F5
:10170000110A5FE0010A5AE0310A55E0100A50E080
:101710007A0A4BE0010A46E0030A41E0010A3CE094
:101720000F0A37E0010A32E0030A2DE0010A28E03F
:10173000070A24E0010A20E0030A1CE0010A18E07D
:10174000190A14E0010A10E0090A0CE0010A08E095
:10175000310A04E0010A40E1AFDA3ED00ADB3CD0B6
:101760002BDB3AD04DDB38D072DB36D08CDB34D07B
:10177000A7DB32D0BFDB30D0D0DB2ED0E9DB2CD0E2
:10178000B8EC0FF029D0DAEC0FF026D0EDEC0FF02A
:1017900023D00DEC10F020D01DEC10F01DD060EC2B
:1017A00010F01AD07BEC10F017D0B9EC10F014D078
:1017B000C9EC10F011D0EEEC10F00ED003EC11F0EB
:1017C0000BD020EC11F008D033EC11F005D05EEC1A
:1017D00011F002D09BEC11F0F7EF1CF0CFEC1BF0F6
:1017E0009E90CD90F00ECF6ECD800001D8906351C9
:1017F00004E6FF0E625D010E635904E2622B000EE7
:1018000063231CD0626B636B050E7C1903E17D5171
:1018100001E18A70010E9E1901E19F5105E0020E5F
:101820009E190CE19F510AE16C516D1107E1897815
:101830008950100B02E0898A01D0899AD8909B5177
:1018400004E6880E9A5D130E9B5904E29A2B000E53
:101850009B2305D09A6B9B6B010E9C6F9D6B8150F7
:10186000DE6EDD6A91EC1AF0141E151E14C0DEFF48
:1018700015C0DDFF91EC1AF0040ED8901532143229
:10188000E804FBE1030E00011414866F876B070E5A
:101890008E1901E18F5101E18ED0060E8E1901E102
:1018A0008F5101E176D0050E8E1901E18F5163E071
:1018B000030E8E1901E18F514AE0020E8E1901E1EB
:1018C0008F5133E0010E8E1901E18F5120E08E51CE
:1018D00001E18F510CE0040E8E1901E082D08F518E
:1018E00001E07FD08651871101E07ED06AD0020EE0
:1018F000861902E1875125E0010E861902E1875120
:1019000054E0030E861970E187516EE168D0030E32
:10191000861902E1875127E08651871152E0010EB6
:10192000861962E1875160E15AD0010E861904E1FF
:10193000875102E1030E56D0020E861904E1875149
:1019400002E1010E4FD0865187114EE13AD0865107
:10195000871104E18C2B000E8D2333D0030E8619E2
:1019600004E1875102E1020E3DD0020E86193CE1EE
:1019700087513AE134D0030E861902E1875128E0FD
:10198000865187111EE0020E86192EE187512CE147
:1019900026D0020E861904E1875102E1070E22D0FB
:1019A000010E861904E1875102E1050E1BD0865114
:1019B00087111AE106D08651871105E18A2B000EA6
:1019C0008B238E6B10D0030E861904E1875102E140
:1019D000060E08D0010E861907E1875105E1040EB5
:1019E00001D0040E8E6F8F6B030E7C1922E17D51A6
:1019F00020E18D518B19E8AE02D08B3504D08A518D
:101A00008C5D8B518D5905E2010E8A6F8B6B8C6B4F
:101A10008D6B8B518D19E8AE02D08D3504D08C5171
:101A20008A5D8D518B5905E28A6B8B6B010E8C6F31
:101A30008D6B020EE15C02E2E16AE552E16E0DEFB0
:101A40001AF0EEEC19F0E6520F0EC112F19ED08E94
:101A5000928216D89EEC1CF0CD92CD96CD88CD9A70
:101A6000CD9CCD90F00ECF6ECE6ACD809F909D80A4
:101A7000F28C8150DF6EF290F28EE5520DEF1AF08B
:101A8000CFEC1BF0FC0E8A129316C70E8912921629
:101A90008998899A8A908A92300E93129284ECD80F
:101AA0001F0E55EC1AF0A5085FE10B0E55EC1AF06D
:101AB00007EC1BF00A0E76EC1CF000011410E66F28
:101AC00015C0E7F00C0E55EC1AF00F0B0001E86F93
:101AD000E96B0E0E55EC1AF0146E07EC1BF00D0EB0
:101AE00076EC1CF000011410EE6F15C0EFF00F0E35
:101AF00055EC1AF00F0B0001F06FF16BE66A94ECF5
:101B000018F0E55200016E6F6F6B010E55EC1AF084
:101B10000001706F716B020E55EC1AF00001766FC8
:101B2000776B030E55EC1AF00001786F796B040E99
:101B300055EC1AF00001686F696B050E55EC1AF050
:101B400006EC1CF0070E55EC1AF0146E156E146AB4
:101B500014C0E6FFE66E060E76EC1CF000011410D1
:101B6000A46F15C0A5F060D000016E6B6F6B6EC0E6
:101B7000E6FFE66A79EC1CF00001706B716B70C0D7
:101B8000E6FF010EE6EC19F0280E0001766F776B88
:101B9000E66E020EE6EC19F0010E2DEC1CF00001D1
:101BA000686B696B68C0E6FF040EE6EC19F0050E81
:101BB00006EC1CF0DFCFE6FF050EE6EC19F00001A5
:101BC000A46B050EA56F320EE66E060EE6EC19F05C
:101BD000E66A070EE6EC19F03CEC1BF0E66A0A0E2A
:101BE000E6EC19F0E66A0B0EE6EC19F0E66A0C0E6C
:101BF000E6EC19F03CEC1BF0A00EE66E0D0EE6ECE8
:101C000019F0860EE66E0E0EE6EC19F0010EE66E89
:101C10000F0EE6EC19F0E66A1E0EE6EC19F0A50EC2
:101C2000E66E1F0EE6EC19F00001B56BB66BB36BF8
:101C3000B46B010EB26F040E8E6F8F6B030E7C6F50
:101C40007D6B7A697B698A908A820001F26BF36B03
:101C500000019A6B9B6BA66BA76BA86BA96B946B2F
:101C6000800E956F926B936B020EE15C02E2E16A6B
:101C7000E552E16E0DEF1AF0080E55EC1AF0000176
:101C8000646F030E6415646F656B42EC1BF001E139
:101C90008B8C010E641903E1655101E18B84020E06
:101CA000641903E1655101E18B80030E641903E1BE
:101CB000655101E18B821200CFEC1BF00401315120
:101CC000DE6EDD6A66EC1AF002E1000E04D0DFEC95
:101CD00019F001E0010E000944E10401100E336F18
:101CE000DFCF35F4AAEC1BF00CE191EC1AF0060EF4
:101CF000145C000E155812E37EEC1CF001E1ED506F
:101D00000DE0F251F31129E0E9EC19F0EE50ED107D
:101D100005E07EEC1CF021E1ED501FE10401346B85
:101D20007EEC1CF011E1ED500FE10001010E6C1989
:101D300001E16D5105E0020E6C1911E16D510FE1E9
:101D4000010E746F756B0BD0DECF6AF0DDCF6BF0D8
:101D5000010E0001F26FF36B02D004013469D1EC83
:101D600019F0020EE15C02E2E16AE552E16E0DEF6C
:101D70001AF066EC1AF002E1000E04D0DFEC19F064
:101D800001E0010E000917E10401110E336F00019B
:101D9000050E7C1906E17D5104E10401050E346F46
:101DA00008D0AAEC1BF003E16CC034F402D06AC086
:101DB00034F4D1EC19F01200AAEC1BF007E1F5ECB9
:101DC0001AF000011410B06F15C0B1F066EC1AF0F3
:101DD00002E1000E04D0DFEC19F001E0010E000971
:101DE0000EE10401200E336F0001B0510401346F85
:101DF000B1C014F0156A1450356FD1EC19F012000F
:101E000066EC1AF002E1000E04D0DFEC19F001E0FC
:101E1000010E00091BE10401210E336F0001AA51DC
:101E2000AB1106E0AC510401346FADC014F006D024
:101E30000001E6510401346FE7C014F0156A145034
:101E4000356F0001AA6BAB6BD1EC19F01200AAEC54
:101E50001BF006E10F0E040131150001AE6FAF6BF0
:101E600066EC1AF002E1000E04D0DFEC19F001E09C
:101E7000010E000907E10401280E336FAEC034F4EF
:101E8000D1EC19F0120066EC1AF002E1000E04D059
:101E9000DFEC19F001E0010E000911E10401290E47
:101EA000336FE6C0ACF0E7C0ADF00001AA69AB6BE0
:101EB0000F0E0001E8150401346FD1EC19F0120087
:101EC000040131510001766F776BE66E020E25EC4E
:101ED0001CF002E1000E04D0DFEC19F001E0010E6D
:101EE000000907E10401300E336F76C034F4D1EC01
:101EF00019F0120066EC1AF002E1000E04D0DFECDB
:101F000019F001E0010E000907E10401310E336F01
:101F100076C034F4D1EC19F01200040131512DECEB
:101F20001CF0040132510001686F696BE66E040E0B
:101F300025EC1CF002E1000E04D0DFEC19F001E00A
:101F4000010E000904E10401320E34EC1CF0120011
:101F500066EC1AF002E1000E04D0DFEC19F001E0AB
:101F6000010E000904E10401330E34EC1CF01200F0
:101F7000040131510001A06FA16BE66E050EE6EC85
:101F800019F0A0C008F0A1C009F0F3EC19F066EC5C
:101F90001AF002E1000E04D0DFEC19F001E0010EAE
:101FA000000907E10401340E336FA0C034F4D1EC12
:101FB00019F0120066EC1AF002E1000E04D0DFEC1A
:101FC00019F001E0010E000907E10401350E336F3D
:101FD000A0C034F4D1EC19F01200F5EC1AF00001B5
:101FE0001410A46F15C0A5F0E850E66E060EE6ECDE
:101FF00019F0A5EC1BF0E66E070E25EC1CF002E1D3
:10200000000E04D0DFEC19F001E0010E000904E13C
:102010000401360E10EC1CF0120066EC1AF002E11E
:10202000000E04D0DFEC19F001E0010E000904E11C
:102030000401370E10EC1CF012000401315118E0BD
:1020400000019E519F1117E19051911109E09451A7
:1020500002E1800E951904E044EC1AF0030E06D05C
:1020600055EC1BF0976B986B996B010E9E6F02D02D
:1020700000019E6B9F6BB351B41102E1000E04D0BE
:10208000DFEC19F001E0010E00090FE10401380E48
:10209000336F65EC1BF005E19F5103E104013469E6
:1020A00002D00401346BD1EC19F065EC1BF005E1B2
:1020B0009F5103E18988898A12008998899A1200C0
:1020C00066EC1AF002E1000E04D0DFEC19F001E03A
:1020D000010E00090FE10401390E336F65EC1BF0AE
:1020E00005E19F5103E10401346902D00401346B1E
:1020F000D1EC19F01200040131511AE10001706BAA
:10210000716B42EC1BF001E18B8C010E641903E151
:10211000655101E18B84020E641903E1655101E10F
:102120008B80030E641912E1655110E18B820ED091
:1021300000017069716B010E6C1901E16D5106E0CF
:10214000020E6C1901E16D5101E08B6A7051E66E6F
:10215000010E25EC1CF002E1000E04D0DFEC19F0BA
:1021600001E0010E000904E104013A0E3BEC1CF011
:10217000120066EC1AF002E1000E04D0DFEC19F058
:1021800001E0010E000904E104013B0E3BEC1CF0F0
:10219000120066EC1AF002E1000E04D0DFEC19F038
:1021A00001E0010E000919E10401410E336F000145
:1021B00091350DE290510008000E915508E29451BE
:1021C0000401346F95C014F0156A145003D0040153
:1021D000346B800E356FD1EC19F0120066EC1AF0FA
:1021E00002E1000E04D0DFEC19F001E0010E00095D
:1021F00009E10401510E336F010E346F050E356F86
:10220000D1EC19F01200010E0401311500016E6FBE
:102210006F6BE66EE66A79EC1CF066EC1AF002E190
:10222000000E04D0DFEC19F001E0010E000907E117
:102230000401600E336F6EC034F4D1EC19F012005B
:1022400066EC1AF002E1000E04D0DFEC19F001E0B8
:10225000010E000907E10401610E336F6EC034F412
:10226000D1EC19F01200CFEC1BF0DE68DD6AA50E90
:102270000401315D09E100016C516D1105E1AEEC25
:102280001BF0A50EDE6EDD6A66EC1AF002E1000EB0
:1022900004D0DFEC19F001E0010E000907E10401B0
:1022A000700E336FDFCF34F4D1EC19F0020EE15C25
:1022B00002E2E16AE552E16E0DEF1AF0CFEC1BF09D
:1022C000A50E0401315D0AE10001050E7C1901E152
:1022D0007D5104E042EC1CF0A50E0FD05A0E040113
:1022E000315D0DE10001050E7C1909E17D5107E129
:1022F0002AEC1BF08A908A925A0EDE6E01D0DE68BC
:10230000DD6A66EC1AF002E1000E04D0DFEC19F091
:1023100001E0010E000907E10401720E336FDFCF07
:1023200034F4D1EC19F0020EE15C02E2E16AE5520C
:10233000E16E0DEF1AF066EC1AF002E1000E04D027
:10234000DFEC19F001E0010E000911E10401730E48
:10235000336F0001050E7C1905E17D5103E1040195
:10236000A50E02D004015A0E346FD1EC19F0120000
:10237000EEEC19F0080EE126B0C0DEFFB1C0DDFFC3
:10238000020EAEC0DBFF030EAFC0DBFF050E000187
:102390006A1901E16B5101E17FD0040E6A1901E174
:1023A0006B516EE0030E6A1901E16B512AE0020ED7
:1023B0006A1901E16B5118E0010E6A1901E16B51D4
:1023C00004E06A5174E16B5172D0050E7C1901E191
:1023D0007D516DE08988899A000EE66EE66AE9EC27
:1023E00019F0D3EC1BF049D0050E7C1901E17D51A9
:1023F0005EE08998898A000EE66EE66AD9CFE9FF29
:102400001ED0050E7C1901E17D5151E0E9EC19F077
:10241000EE500001E65DEE50E759EE50E859EE50FF
:10242000E95913E2E9EC19F0F0EC1BF0D6EC1AF0E4
:102430008998898A000E69EC1BF0040FE96EDACFE7
:10244000EAFFD3EC1BF0010E18D0E9EC19F0EE50C6
:10245000E65D146EEE50E759156EEE50E859166EB3
:10246000EE50E959D6EC1AF08988899A000E69EC89
:102470001BF0040F1CEC1AF0000E7FEC1AF017D0C2
:10248000DFCFE6F0010EDBCFE7F0020EDBCFE8F0A6
:10249000030EDBCFE9F00BD0DFCFEEF0010EDBCF88
:1024A000EFF0020EDBCFF0F0030EDBCFF1F065ECC6
:1024B0001BF005E19F5103E18988898A02D0899840
:1024C000899A080EE15C02E2E16AE552E16E0DEFE5
:1024D0001AF0EEEC19F00A0EE1260001905191116C
:1024E00001E1EDD0030E9E1901E0E9D09F5101E01A
:1024F000E6D09851945D146E9551995514C0DEFF45
:10250000DD6E91EC1AF00001800E15140CE00868E5
:102510000968DECF0DF0DDCF0EF0A8EC23F006C089
:10252000DEFF07C0DDFF91EC1AF00001A351151882
:10253000E8AE02D0153404D01450A25D1550A35952
:1025400001E3D7D09651945D146E9551975514C000
:10255000DEFFDD6EA4C018F0A5C019F01A6A1B6A70
:1025600019AE02D01A681B6891EC1AF0166A176A45
:1025700015AE02D01668176814C006F015C007F033
:1025800016C008F017C009F018C00BF019C00CF005
:102590001AC00DF01BC00EF0E0EC25F002C006F0F2
:1025A00003C007F004C008F005C009F0000E066C77
:1025B000071E0722081E0822091E09220B6A0C6A40
:1025C000010E0D6E0E6A74EC23F0060E06C0DBFFE2
:1025D000070E07C0DBFF080E08C0DBFF090E09C0AD
:1025E000DBFFD950060F02EC1CF00001EA51EE248B
:1025F000146EEB51EE20156EEC51EE20166EED517F
:10260000EE20176EE8EC1AF09AEC1CF0F0EC1BF0E0
:10261000176E060E14C0DBFF070E15C0DBFF080E99
:1026200016C0DBFF090E17C0DBFF89EC1BF0080E9C
:10263000DBCF16F0090EDBCF17F014501510161073
:10264000171057E094C098F095C099F0D950060F34
:1026500002EC1CF0D890030EEB50000A03E6000ECB
:10266000DCEC1BF024E2060EDBCF06F0070EDBCF1E
:1026700007F0080EDBCF08F0090EDBCF09F00B687E
:102680000C680D680E68E0EC25F0060E02C0DBFF5A
:10269000070E03C0DBFF080E04C0DBFF090E05C0F8
:1026A000DBFF8988899A19EC1CF0000E05D0899807
:1026B000898A19EC1CF0010E7FEC1AF018D09051A9
:1026C000911117E0945102E1800E951912E0010E6C
:1026D0009E1905E19F5103E144EC1AF005D0020E6A
:1026E0009E1907E19F5105E1030E9E6F9F6B89883C
:1026F000898A0A0EE15C02E2E16AE552E16E0DEFC1
:102700001AF0EEEC19F0060EE1267AC014F07BC048
:1027100015F0166A176A15AE02D016681768E8EC4D
:102720001AF000018D518B19E8AE02D08B3504D020
:102730008A518C5D8B518D5908E28C518A5D8A6F6C
:102740008D518B598B6F8C6B8D6B8B518D19E8AEC6
:1027500002D08D3504D08C518A5D8D518B5908E2A1
:102760008A518C5D8C6F8B518D598D6F8A6B8B6B01
:10277000040E8014040818E1050E7C1901E17D5156
:1027800013E08A518B1110E08A07000E8B5B898859
:10279000899A1FEC1CF0000E7FEC1AF065EC1BF020
:1027A00021E19F511CE01ED0040E801404081CE19E
:1027B000050E7C1901E17D5117E08C518D1114E05B
:1027C0008C07000E8D5B8998898A1FEC1CF0010E26
:1027D0007FEC1AF065EC1BF005E19F5103E189885D
:1027E000898A02D08998899A80B404D1DE6ADD6A28
:1027F000040E801412E182EC1CF004E6280E145C36
:10280000000E15580AE2190EE66E56EC26F0E55257
:10281000DF2A010EEDE3DB2AEBD782EC1CF004E6A5
:10282000020E145C000E155801E2E4D000018C6B1E
:102830008D6B8A6B8B6B82EC1CF004E6280E145CAB
:10284000000E15584EE2050E7C1901E17D5101E1A3
:10285000D1D0010E7C5F000E7D5B030E7C17000E55
:102860007D177C517D1103E1010E7A6F7B6B010EA8
:102870007C1905E17D5103E10A0E7A6F7B6B020E34
:102880007C1905E17D5103E1640E7A6F7B6B030EC9
:102890007C1904E17D5102E17A697B69010E7C15A6
:1028A000146E156A7CC016F07DC017F0D8901732F0
:1028B0001632010E1616000E14501618E8B081805C
:1028C000E8A081907CC014F07DC015F0D89015323E
:1028D0001432010E1414E8B08182E8B08BD08192DA
:1028E00089D07C517D110EE180B408D06251400B3B
:1028F00003E08A908A92F8D78A80F6D78A908A92E3
:102900009DDA73D0010E7C1911E17D510FE180B485
:1029100008D06251400B03E08A908A92F8D78A80EF
:10292000F6D7AEEC1BF042EC1CF064D0020E7C1922
:1029300037E17D5135E19E519F110FE080B408D001
:102940006251400B03E08A908A92F8D78A80F6D7CA
:102950009E6B9F6B8998899A21D080B408D0625170
:10296000400B03E08A908A92F8D78A80F6D790517C
:1029700091110DE0945102E1800E951908E044ECAC
:102980001AF0030E9E6F9F6B8988898A07D055ECD9
:102990001BF0800E976F010E9E6F9F6B8A8012D086
:1029A000030E7C1911E17D510FE180B408D0625112
:1029B000400B03E08A908A92F8D78A80F6D73CECE5
:1029C0001BF08A908A8216D0050E7C1911E17D5188
:1029D0000FE180B408D06251400B03E08A908A92E4
:1029E000F8D78A80F6D72AEC1BF08A908A9202D018
:1029F00080A4FED7060EE15C02E2E16AE552E16ED8
:102A00000DEF1AF0EEEC19F0060EE126ECEC1BF0DF
:102A100002E1010E01D0020E00016C6F6D6BDE6AE7
:102A2000DD6A7051711116E042EC1BF001E18B8CF4
:102A3000010E641903E1655101E18B84020E6419F2
:102A400003E1655101E18B80030E641903E16551D7
:102A500001E18B82726B736B86EC1CF022E190ECCF
:102A60001BF06851141802E1695115183DE0010E80
:102A7000DE6EDD6A88EC1AF019EC1BF015AE02D0A0
:102A8000166817682CEC1AF02FE282AE2DD00001E8
:102A90006851691102E148D901D04ED959EC1AF0B8
:102AA000EBD760EC1AF020E1ED501EE190EC1BF04A
:102AB0006651141802E16751151816E088EC1AF0F7
:102AC00019EC1BF015AE02D0166817682CEC1AF042
:102AD0000BE282AE09D0ECEC1BF002E12DD901D063
:102AE00023D959EC1AF0ECD70001030E7C190AE146
:102AF0007D5108E160EC1AF005E1ED5003E1010EB3
:102B0000726F01D0726B736B88EC1AF0F90EDBCF29
:102B100014F0FA0EDBCF15F0FB0EDBCF16F0FC0E37
:102B2000DBCF17F02CEC1AF001E37DD082AE7BD026
:102B3000ECEC1BF015E0E60EE96E000EEA6E00010B
:102B4000EE51EE5CEF51EE58F051EE58F151EE5867
:102B50006AE2E62B000EE723E823E923E5D812D04A
:102B60000001E651E711E811E91106E0E607000E61
:102B7000E75BE85BE95B05D060EC1AF054E1ED50EF
:102B800052E1DAD8FD0EDBCF66F0FE0EDBCF67F048
:102B900086EC1CF007E100017451751103E0746BC1
:102BA000756B41D060EC1AF005E1ED5003E1040EC5
:102BB000801439E060EC1AF027E1ED5025E10001C6
:102BC000030E7C1921E17D511FE1ECEC1BF007E1C4
:102BD0008D3505E28C510008000E8D5510E3D9505B
:102BE000FD0F28EC1CF0010EEE180EE1ED500CE18B
:102BF0008B350AE28A510008000E8B5505E28A6B7C
:102C00008B6B8C6B8D6B0FD0F7EC1CF0200E0001E2
:102C1000B85D03E16D50020B03E086EC1CF003E0AD
:102C200059EC1AF073D70001725173111AE0B80E03
:102C30008B166451651101E18B8C010E641903E15F
:102C4000655101E18B84020E641903E1655101E1D4
:102C50008B80030E641903E1655101E18B82FCEC6A
:102C60001BF00001726B736B9E519F1134E0D950C1
:102C7000F70F28EC1CF0020EEE1801E1ED502BE0EE
:102C80009051911128E0020E9E1901E19F5105E03B
:102C9000030E9E1920E19F511EE1ECEC1BF00EE1AA
:102CA000F90EDB500001EA5FFA0EDB50EB5BFB0E26
:102CB000DB50EC5BFC0EDB50ED5B0DD0F90EDB5016
:102CC0000001EA27FA0EDB50EB23FB0EDB50EC236E
:102CD000FC0EDB50ED237DDB010EEE1817E1ED500D
:102CE00015E188EC1AF019EC1BF015AE02D016684D
:102CF0001768B2DB0BE282AE09D00001685169119E
:102D000002E11AD801D010D8D4DBEDD70001705100
:102D1000711101E08B6A6C6B6D6B060EE15C02E277
:102D2000E16AE552E16E79D300016E516F1102E163
:102D3000A4EF16F0E2EF16F000016E516F1102E100
:102D4000E2EF16F0A4EF16F0030E0001641901E1A2
:102D5000655123E0020E641901E1655116E0010E90
:102D6000641901E165510AE0645120E165511EE1F9
:102D70004EEC1CF01BE18B9C8B8414D054EC1CF0AB
:102D800015E18B9C8B948B800ED05AEC1CF00EE1DD
:102D90008B9C8B948B908B8207D060EC1CF006E1AF
:102DA0008B8C8B948B908B92FCEC1BF0010E0001B2
:102DB0006425646F000E6521656F030E6417000EB5
:102DC00065171200030E0001641901E1655123E04B
:102DD000020E641901E1655117E0010E641901E169
:102DE00065510CE0645120E165511EE160EC1CF07E
:102DF0001BE18B9C8B948B908B8214D04EEC1CF03F
:102E000013E18B8C8B9405D054EC1CF00DE18B9C62
:102E10008B848B9006D05AEC1CF006E18B9C8B9433
:102E20008B808B92FCEC1BF00001010E645F000EA6
:102E3000655B030E6417000E65171200CFDA0A0EE9
:102E4000E126E6C0DFFF010EE7C0DBFF020EE8C0AF
:102E5000DBFF030EE9C0DBFFBCDAD8803F0EEE5487
:102E6000420EEE540F0EEE54000EEE5409E23F0EE9
:102E7000DE6E420EDE6E0F0EDE6EDD6ADD52DD525C
:102E8000010E67DB080EDB6A090EDB6A8AEC1CF0B8
:102E900002E3020E5EDB8EEC1CF002E3030E59DB54
:102EA000E0EC1BF005E3040EF36EDB6E050EDB6A4F
:102EB000E6EC1BF002E3050E4CDB8BDAD4DB02E31D
:102EC000060E47DB81DBFEE16351010BFDE0060EE0
:102ED000DB6A070EDB6A89EC1BF0040EDBCF16F011
:102EE000050EDBCF17F015501718E8AE02D01734D7
:102EF00004D01650145C1750155807E2CCD8060EB3
:102F0000DB2A070EE8E3DB2AE6D780A4FED780B4ED
:102F1000FED75ADBFEE16351010BFDE05ADAA3DB79
:102F20000AE357DAA00EEE5E860EEE5A010EEE5A56
:102F3000000E9CDAF3D77ADA09E080A4FED780B4D9
:102F4000FED742DBFEE16351010BFDE0E6EC1BF036
:102F50000CE3E6EC1BF00CE33CDA100EEE5E270E01
:102F6000EE5A000EEE5A82DAF4D760DA01E0A3D806
:102F70005DDA09E080A4FED780B4FED725DBFEE150
:102F80006351010BFDE0E0EC1BF00CE3E0EC1BF007
:102F90000CE31FDAE80EEE5E030EEE5A000EEE5A58
:102FA00065DAF4D743DA01E086D840DA09E080A494
:102FB000FED780B4FED708DBFEE16351010BFDE0D4
:102FC0008EEC1CF008E38EEC1CF008E302DA640ED1
:102FD00066EC1CF0F8D72ADA01E06DD827DA09E0B0
:102FE00080A4FED780B4FED7EFDAFEE16351010B77
:102FF000FDE08AEC1CF008E38AEC1CF008E3E9D958
:103000000A0E66EC1CF0F8D711DA01E054D80EDA9B
:1030100009E080A4FED780B4FED7D6DAFEE1635182
:10302000010BFDE0D6D9EECF14F0EECF15F0EECFC8
:1030300016F0EFCF17F0145015101610171013E0FC
:10304000C8D9D880000EEE54000EEE54000EEE5497
:10305000000EEE5409E2BDD9EE06000EEE5AEE5A0D
:10306000EE5A21D8EDD727D8AFDAFEE16351010B34
:10307000FDE08A8080A4FED780B4FED78A90A4DACF
:10308000FEE16351010BFDE00A0EE15C02E2E16A40
:10309000E552E16EC2D198DAFEE18A806351010BFC
:1030A000FDE08A90120090DAFEE18A826351010B02
:1030B000FDE08A92120088DAFEE18A826351010BF8
:1030C000FDE06351010BFDE16351010BFDE08A92CC
:1030D0001200D9CFE6FFE1CFD9FF020EE126FE0EA6
:1030E000DB50A96EFD0EDB50A86EA69EA69CA684A2
:1030F000F250DE6EDD6AF26A550EA76EAA0EA76E5A
:10310000A682DF50F26E0000A1B802D00000FCD70A
:10311000A694A198020EE15C02E2E16AE552E16E3A
:10312000E552E7CFD9FF120059D9FE0EDB50A96E48
:10313000A69EA69CA680A85070D16DA205D00001C5
:103140006051611113E01BD00001B8510BE0B805CC
:1031500009E0020EB85D06E0040EB85D03E0100E53
:10316000B85D06E100016051611109E18986120034
:10317000200EB85D07E100016051611102E18996FE
:1031800012008986120012001200120012008AEF4B
:1031900024F012001E0EE66E010EE66E1DEC21F00C
:1031A000E552E552EED26D840001080EFE6F070E67
:1031B000FF6FFE07000EFF5BFE51FF11FAE16D94F9
:1031C0001200D9CFE6FFE1CFD9FFFD0EDBCF08F02B
:1031D000FE0EDBCF09F0720E081801E1095033E052
:1031E000E868081802E17F0E09182BE0740E081831
:1031F00001E1095024E0750E081801E109501DE0B5
:10320000730E081801E1095016E0030E081801E1D9
:1032100009500FE0020E081801E1095008E0010E04
:10322000081801E1095001E010D0B4DF0FD0B1DF80
:103230000DD0ADDF0BD0A9DF09D0A5DF07D0A4DF0B
:1032400005D0A4DF03D0000001D000D0010E00D0D3
:10325000E552E7CFD9FF1200C1D8E652DF6A040178
:103260002351030A0BE0010A0AE1225108E1DF6A57
:10327000DF50030804E374D9DF2AFAD72251E5525C
:10328000CCD0ACD8030EE126DF6A010EDB6A020E59
:10329000DB6A0001B751740A2AE0060A36E1B5512B
:1032A000B61102E1000E03D02DDA01E0010E000993
:1032B0002CE1B5C0E9FFB6C0EAFFEE52EF50E66E72
:1032C00071D9E552E750EE6EED6A6CD9000ED880E8
:1032D000EE54000EED5419E2DF50030805E340D927
:1032E000FBDAEF6ADF2AF8D70001740E0DD0B35174
:1032F000B41102E1000E03D062D801E0010E000912
:1033000004E14FD80001720EB76F030EE15C02E2D8
:10331000E16AE552E16E81D004012351030A06E01F
:10332000010A08E1225101E1020C000C225101E1E5
:10333000030C000C000C0401230508E1225110E1EC
:103340000001300EC96F040E97EF1BF0030E235DD2
:1033500007E1225105E10001000EC96F050EE7D912
:103360001200DADF030A10E0010A01E01200040192
:10337000225116E126C4D1F027C4D2F00001300E4C
:10338000CE6F040E9EEF1BF00401225109E126C40A
:10339000D1F027C4D2F00001000ECE6F050ECED9B9
:1033A0001200040EE66E330EE66E040EE66E010E9B
:1033B000E66EB8DAF3CFB3F0F4CFB4F0E2D1B3C035
:1033C000E9FFB4C0EAFFEF50800B1200E66E79EF20
:1033D0001CF0D9CFE9FFDACFEAFF1200D9CFE6FF20
:1033E000E1CFD9FF1200F4EC22F007C014F008C0BE
:1033F00015F009C016F00AC017F0CD0E0C6ECC0EF9
:103400000D6E0E6E410E0F6E07EC23F0D5EC23F01F
:1034100008C0A2F009C0A3F01200E552E7CFD9FF1F
:103420001200EAD90001725173111200D950080F2D
:10343000E9D9EE50ED101200E5D9D3EF1BF0E66E9E
:10344000E66A9DEC25F0E552E5521200EE58000EBA
:10345000EE58000EEE5812006DDA1450EE5C155066
:10346000EE581650EE581750EE581200EE5A1BDE6A
:10347000010EF36E080EF3CFDBFF090EDB6A1200BC
:10348000E7D9EE50ED101200E6C0EAF0E7C0EBF02D
:10349000E8C0ECF0E9C0EDF094C096F095C097F06C
:1034A00094C098F095C099F01200E66E3DDEE552AA
:1034B000120040DAEE2A000EEE22EE22EE22120078
:1034C000D950F70FC5D9010EEE1812000001B35103
:1034D000B4111200DACFE4FFE2CFDAFFE9CFE4FF64
:1034E000EACFE4FFF6CFE4FFF7CFE4FFF5CFE4FF48
:1034F000F3CFE4FFF4CFE4FFFACFE4FF1200E66E6F
:10350000E66A02EC15F0146E080EE15E145012002B
:10351000020EDB6A030EDB6A040EDB6A050EDB6A51
:103520001200DECF14F0DDCF15F01200E5CFFAFF68
:10353000E5CFF4FFE5CFF3FFE5CFF5FFE5CFF7FFEC
:10354000E5CFF6FFE5CFEAFFE5CFE9FFE5CFDAFF0C
:103550001200F36E040EF3CFDBFF050EDB6A1200E0
:10356000BBD9EF50E66EDF50EA6A330FE96E040E06
:10357000EA22E552E750EF6E1200010EDB50EA6AD4
:10358000F40FE96E000EEA2212002CEC08F0550E42
:10359000E66EBCEC08F0E5521200E66E90EC08F026
:1035A000E5521200D950010F02EF1CF0176E040E05
:1035B00014C0DBFF050E15C0DBFF060E16C0DBFFD7
:1035C000070E17C0DBFF120000016351010B120050
:1035D000020E14C0DBFF030E15C0DBFF040E16C085
:1035E000DBFF050E17C0DBFF120032C414F014C05D
:1035F00015F0146A000E1416FF0E15160401315151
:103600001200320EE66E56EC26F0E5521200156EF0
:10361000146A000E1416FF0E151614C0E6FF15C02E
:10362000E6FF1200E552E7CF15F0E552E7CF14F0C0
:10363000120078C014F079C015F0166A176A1200EB
:1036400014C015F0146A010E14C0DBFF020E15C081
:10365000DBFF12003CEC0EF000017C6B7D6B010E79
:103660007A6F7B6B1200A00EEE5C860EEE58010E98
:10367000EE58000EEE5812000001E66BE76BE86BA7
:10368000E96B1200B80E8B16941664516511120086
:10369000DBCFF4FFF350F45C1200E66E010EE66E31
:1036A0009DEC25F0E552E55212000001EA6BEB6B50
:1036B000EC6BED6B0001966B12008B6A8A908A921C
:1036C000050E00017C6F7D6B12000001030E9E1938
:1036D0001200E66EE66AD9501200030E14C0DBFF3A
:1036E000040E15C0DBFF1200030EDBCF14F0040E36
:1036F000DBCF15F01200030E08C0DBFF040E09C07B
:10370000DBFF1200B5C0E9FFB6C0EAFFEF50800B47
:103710001200060EDBCF14F0070EDBCF15F01200FF
:10372000FD0EDBCF14F0FE0EDBCF15F01200CA6FDA
:10373000040ECC6FCD6BC10ECB6F1200CF6F580E45
:10374000D36F320ED46FD08F1200A5C014F0156A5B
:10375000145012000001F251F31112000001E65161
:10376000E66E0A0E33DEE7C014F0156A1450E66EFA
:103770000B0E2CDE0F0E0001E815E66E0C0EE6EFC8
:1037800019F0400EE66E300EE66E040EE66EE66A46
:10379000010EC8D8F3CFB5F0F4CFB6F012001EDE9C
:1037A000020EE1261200EECFE6FFEECFE6FFEECFEF
:1037B000E6FFEFCFE6FF1200EE5C000E26EF1AF0F8
:1037C00008DEE80EEE5C030E26EF1AF002DE100EA5
:1037D000EE5C270E26EF1AF0D950FD0F40EF1AF0DD
:1037E000E651EE5C146EE751EE58156EE851EE5856
:1037F000166EE951EE58120076C0E6FF83EC26F013
:10380000E5521200E96EDACFEAFF1200DE6EDD6AE1
:10381000000EDFCF08F0010EDBCF09F0F3EF19F057
:10382000336F0001A4510401346F8FDF356FD1EF86
:1038300019F0E7DE020E4DDF060F1CEF1AF0E1DE95
:10384000010E47DF020F1CEF1AF0C0DD66EF1AF021
:10385000E96EFF0EDA20EA6E12000001786F796BD4
:10386000E66E030EE6EF19F0336F78C034F468C0EB
:1038700035F4D1EF19F0336F000170510401346F4A
:10388000D1EF19F064C0E6FF080EA0DD5DEF1BF07C
:10389000A5DDE652F29E9290809012008B8C8B8474
:1038A0008B908B9211EF1AF08B9C8B848B808B9278
:1038B00011EF1AF08B9C8B948B808B8211EF1AF096
:1038C0008B8C8B948B908B8211EF1AF0EE5E000E36
:1038D000EE5AEE5A36EF1AF0DF50EA6A300FE96E10
:1038E000040EEA221200ABDD16EF08F0DEDD12EF67
:1038F0001BF069EC18F0E552E55212006ADDFF0E8C
:10390000EE1812000EDED89015501200D950F70FA5
:1039100040EF1AF05EDD0A0EDCEF1BF05ADD640E9C
:10392000DCEF1BF0E66E4DEC21F0146E050EE15E4F
:0C39300014501200D950020F02EF1CF0DE
:04393C00B9EC22F0D0
:10394000A09A6A6A686A706A08EC22F055EC22F064
:10395000DF6A3EEC22F003E2F8EC21F0FAD76D8C3E
:103960006E6A6D986D9C68A607D068960001CB6B57
:10397000D06BD16BD26BF7D70001010EE26FE36F12
:10398000E46BE56BD86BDF6A020EDF5C1AE2EA6A71
:10399000DF34BCEC22F0EA22EE6AED6AEA6ADF3438
:1039A000C3EC22F0EA22EE6AED6ADF50D6EC22F098
:1039B000EA22EF6ADF50D1EC22F0EA22EF6ADF2A36
:1039C000E3D70001080EC36F040EC46F160E706EAD
:1039D0000401200E026F040E036F080E016F840EA7
:1039E000006F0001B96BB86BE552D2EF21F0B9EC72
:1039F00022F00001B80507E16DBA05D0686A698058
:103A00006988020EB86F6850040B05E06950040B1A
:103A100002E0689491D86DB23ED06850010B09E085
:103A20006950010B06E08ADFA08A0001040EB86F1E
:103A300068906850100B05E06950100B02E071D8D7
:103A4000689868AC08D069AC05D05CEC22F0730EC5
:103A5000BFEC21F0689C6850200B04E06950200BFB
:103A600001E04CD86850020B0BE06950020B08E0F3
:103A70005CEC22F0E6687F0EE66ECAEC22F06A6A21
:103A8000040E0001E76EB819E8AE02D0E73402D0A8
:103A9000E750B85D02E2A19A2ED069A62BD0DF6A6A
:103AA000040EDF5C27E268A625D06CCFD9F00001B8
:103AB000D951780BE842E842E842DA6F6896D9B506
:103AC00004D0DA51D1EC22F003D0DA51D6EC22F056
:103AD000EA22EF70DA5102E13DD80AD0000EE66E1C
:103AE000E66AD90EE66E000EE66E720EBFEC21F0AD
:103AF000DF2AD6D7A19AE552D2EF21F070A00FD0DD
:103B0000DEEC21F0EF50800809E1C8EC21F0EF5025
:103B1000840804E1DEEC21F08C0EEF6E7090689A60
:103B20001200698468986D820001010ED86F24EC40
:103B300022F0750EBFEF21F00001D86B24EC22F0CB
:103B4000740EBFEC21F06D92699468A402D0689461
:103B5000FCD71200B9EC22F0FD0E0001D91540E1AE
:103B60007E0ED915E8407F0B040DF3CFBBF0F4CFE8
:103B7000BCF0000EBB27040EBC23BBC0BDF0BCC014
:103B8000BEF0BD75DEEC21F0EF503C0BE842E842A0
:103B90000D0824E1DF6A080EDF5C1AE2DEEC21F09A
:103BA000020EE926000E11EC22F0EF50E66EDF5017
:103BB000EA6A200FE96E040EEA22E552E750EF6E42
:103BC000DEEC21F0E9EC22F0EE2AEF22DF2AE3D747
:103BD000DEEC21F089EC22F00AD807D025D805D0F8
:103BE000FD0ED915040801E12ED8E552DBD3000102
:103BF000C76BE16BE46BE56BDB6BC86BC9DBEF9EFE
:103C0000C375C6DBEF9EC37578EC22F0EF9ECB6BDD
:103C1000CC6BCD6BD06BD16BD26B50D824EC22F037
:103C2000030EADDBEDEF1FF0020E0001C85D02E1F7
:103C300059EF20F0C86BDB5104E198DB8C0EEF6E7E
:103C40001200DB6B1200B9EC22F0A2DBEF50400B4C
:103C500001E0010EDF6E0001C375080EB85D08E1DA
:103C600022C46EFF6E5002E0100E01D0040EB86F39
:103C7000C80513E18DDBA7DBDDD9020E0001C75DAE
:103C800003E186DB840E07D0DF5003E181DBC80E41
:103C900002D07EDB880EEF6E0FD0D0AF0CD0D351A8
:103CA000D41107E005D0D4C0FAFF0001D351F96E5A
:103CB000FADF0001D09FC86BE55274D30401205194
:103CC000600BE842E842E842E842E842000901E0CD
:103CD000120021510C0A45E00B0A3FE00C0A31E0CA
:103CE000010A22E00B0A1EE0020A1CE0030A18E0A7
:103CF000080A10E0010A0CE00F0A08E0030A01E0DC
:103D000012000001CB8F080EB86F120077EF1FF082
:103D1000BDEF20F00001B90EC96F000ECA6F0CD0C4
:103D2000B4EF1FF0B2EF1EF024510001C96FCA6B4F
:103D3000BA0EC927000ECA23CB81010ECC6FCB8FE0
:103D400012000001CB8F04012451EA6ABA0FE96E18
:103D5000000EEA2222C4EFFF120076DB020EBFEF54
:103D600021F012001ADB030EE1260401220510E106
:103D700020511F0B00090CE10001CB8F030E040141
:103D8000215D04E10001010ED76F02D00001D76B65
:103D90000401225163E120511F0B02085FE124510D
:103DA0000F0B00095BE024510F0B010857E3200EB5
:103DB0000001B85D53E1CB8F040124BF04D0C4DB04
:103DC00049DB4EDB03D0C5DB45DB4EDBEA22020ECE
:103DD000EFCFDBFF78DB010B03E1000EDF9401D0B6
:103DE000DF8424BF02D0B0DB01D0B3DBEA22DECF18
:103DF000EEFFDDCFEDFF030E215D0CE1DCDB07E024
:103E000024BF02D02DDB01D02FDBEA22EF82840E0B
:103E1000E5DB24D0DF74CFDB06E0B5DAEF9EB3DA62
:103E2000EF8C81DB02D0AFDAEF8CDF744CDB020B5E
:103E300006E1C1DB11E0A7DAEF50040B0DE104014C
:103E400024BF02D00DDB01D00FDBEA22EF923B0E44
:103E5000146EB5DB68DB02D03B0EB1DB030EE15C18
:103E600002E2E16AE552E16E9DD20001E25121E1F8
:103E7000010EE26FE3511DE1010EE36F020EC85D1A
:103E800007E186DAEE52EF6A83DAC80EEF6E1200AF
:103E9000C8050FE1DB6B92DAEE52080EEF6E8EDA98
:103EA00038DB8CDA840EEF6E010EDB6F5FDA800E8A
:103EB000EF6E12000001E46BE56B020EC85D04E1D9
:103EC00082DB81DA15DB10D0CC510401265D0001C4
:103ED000CD510401275904E226C4CCF027C4CDF00B
:103EE000A9D856DA70DA54DAC80EEF6E1200800ED6
:103EF0000401205D38E10001C00ECB6F04012351A5
:103F0000030A1AE0010A09E0030A2BE10001E40EAA
:103F1000C96F490ECA6F120E1ED0E3DA940EF62650
:103F20004A0EB4DA020E0001D5DAF5CFCCF0030E5A
:103F3000D1DAF5CFCDF01200030E225D0FE2D1DA17
:103F4000960EF6264A0EA2DAC9C0F6FFCAC0F7FFDF
:103F50000800F5500001CC6FCD6B12000001CB6B57
:103F600012000001CB6B1200DADA0401286B296B16
:103F700020511F0B020A11E0030A0CE0010A1CE1A8
:103F80000001CB8F040128810001D70515E1040150
:103F9000288312D00001CB8F0FD00001CB8F0401FA
:103FA00024BF02D0D1DA01D0D4DA54DAECD9EF5000
:103FB000040B02E0010E286F0001CBAF07D0280EE2
:103FC000C96F040ECA6FCB81020ECC6F020EE15C8A
:103FD00002E2E16AE552E16EE5D16D980001CBBFE6
:103FE0000DD0D0AF09D0020EC86FE55101E162DFFC
:103FF0000001E36BE26B12009DEF22F0040120AFA1
:104000000DD00001010EC86FE45101E153DF000142
:10401000E36BE26BE1510DE135EF1FF00001020EA1
:10402000C86FA4D9840EEF6EE36BE26BE15101E13E
:104030001CDF12009EDA080EDF6E0001CC5D000E60
:10404000CD590AE2CCC0DFFFC75102E1010E03D017
:10405000C70502E1020EC76FDF50156AE850CC5D5C
:10406000CC6F1550CD59CD6F93D9EE52DFCFEFFF06
:10407000280ED56F040ED66FCBB10DD0DF5017E0F0
:10408000C9C0F6FFCAC0F7FFC92B000ECA2308003B
:10409000F550CDD9F3D7DF500AE0C9C0E9FFCAC057
:1040A000EAFFC92B000ECA23EF50C1D9F4D7E5525D
:1040B00079D135DA83D9EE52EFCFDFFFDFCF14F0BD
:1040C00014500001D15D000ED25902E2D1C0DFFFD1
:1040D000DF50146E156AE850D15DD16F1550D2597A
:1040E000D26F010EDB6ADF50F36E010EDBCFF4FFFF
:1040F000F350F45C16E2010EDB50EA6A280FE96E19
:10410000040EEA22EF50E66ECEC0E9FFCFC0EAFF10
:10411000CE2B000ECF23E552E750EF6E010EDB2AC7
:10412000E2D7000ED880D155000ED2550DE24BDA01
:104130004AD944D9EF50400B03E1DAD9C80E02D076
:10414000D7D9880EEF6E12D011D9840EEF6ED351ED
:10415000D41107E005D0D4C0FAFF0001D351F96EA5
:10416000FADF0001D09FE15101E17FDE020EE15C48
:1041700002E2E16AE552E16E15D1FBD90001CB8F75
:1041800047D9DF6A7BD902E233D9FCD76D8C010EA7
:10419000E66EE66AE66ABA0EE66E000EE2D96D9C3D
:1041A0000001080EC36F040EC46F000EBB6F040E37
:1041B000BC6FBBC0BDF0BE6F22C4B9F0B95102E103
:1041C000100E0BD0010EE66EE66AB90EE66E000E1A
:1041D000E66E010ED4D80001200EB86FE552E2D091
:1041E0009ED9000EDE6E040EDD6EF3D8040DF4CF02
:1041F00015F0D9CFE9FFDACFEAFFF350EE261550DC
:10420000ED22C1D8EF9EFD0EDB5002E1ECD801D0CB
:10421000B1D8EA22DECFEEFFDDCFEDFFB4D8EF9CC0
:10422000B2D8040EE926000EEA22EF8C020EE15C01
:1042300002E2E16AE552E16EB5D071D9FD0EDBA470
:1042400002D0E66A2BD9FD0EDBA203D0010EE66E8A
:1042500025D9FE0EDB50156A700F146E0F0E08D9AB
:1042600092D8FD0EDBCFEFFF020EE15C02E2E16AC5
:10427000E552E16E97D053D9FE0EDB5002E15DD9D5
:1042800005D0A7D83AD9A5D8010F37D9020EE15CDD
:1042900002E2E16AE552E16E85D041D9FD0EDB50C4
:1042A00002E068D801D09FD8D5D8D9CFE9FFDACFBE
:1042B000EAFFEE50ED1003E1F36AF46A21D063D80F
:1042C00088D9FB0EDBCFEEFFFC0EDBCFEDFF5BD81A
:1042D000EE52FA0EDBCFEFFF400E71D9880E7ED979
:1042E000FD0EDB5002E046D801D07DD8EA22EF7403
:1042F000DECF14F0DDCF15F014C0F3FF15C0F4FFCE
:10430000020EE15C02E2E16AE552E16E4BD045D873
:104310006DA812D023D9400EEE16EE6AEE6AEE6A50
:104320001DD9EE7C27D8EA22EF74400E146E16D900
:104330001450EF1613D9EF7C35D06D6A696A00010D
:10434000B86B12000001B85110E180A20ED06D6A66
:10435000696AABD8D08EA28AA08AF28E6DB602D0DE
:104360006D86FCD70001010EB86F12002CD9D1D890
:1043700078EF22F0FE0EEA6ADB34BCEF22F0E66E44
:10438000E66ACAEF22F0DECFE9FFDDCFEAFF1200D6
:10439000C3C0E9FFC4C0EAFF1200D9CFE6FFE1CFF6
:1043A000D9FF1200E552E7CFD9FF120024510F0BBD
:1043B000E96EEA6AD890E936EA361200BBC0E9FF36
:1043C000BCC0EAFF120005D9280EEE6E040EED6E99
:1043D0001200FD0EDB50E824166EFE0EDB50040DBD
:1043E000F35016241200FE0EEA6ADB34C3EF22F00B
:1043F000DF50040DF3CFE9FFF4CFEAFF000EE9260A
:10440000040EEA22EE6AEE6AEE6AEE6ADF2A120013
:10441000010EE66EE66AE66A710EE66E0F0EB1EF09
:1044200022F0EA22EE50EFCFEAFFE96E1200E66ECC
:10443000D5C0E9FFD6C0EAFFD52B000ED623E55242
:10444000E750EF6EDF061200000EE66EE66AE66EDB
:10445000E66A1200EA22EECFDEFFEDCFDDFF1200AA
:1044600024510F0BD1EF22F024510F0BD6EF22F085
:10447000152214C0DEFF15C0DDFF1200DF50146EE0
:10448000156A080E145C000E15581200F722090078
:10449000F5CFC9F00A00F5CFCAF01200FE0EDBCF4F
:1044A000E6FF9EDEE552E5521200160E6F6E9F0E7D
:1044B0006B6E7B0E696E1200010EE66EE66A000EF0
:1044C000E66EE66A1200D950020FE96EDACFEAFF13
:1044D000EF501200F76AC925F66ECA51F72208009C
:1044E00012002251F66EF76AD890F636F7361200AF
:1044F000BDC0E9FFBEC0EAFF1200040DF3CF14F007
:10450000F4CF15F0000E1426040EB2DF840EEEEF89
:1045100022F05FD8200EEE6E040EED6E12003DDF2D
:10452000020EE1261200020EE66EE66ADECFE6FF1C
:10453000DDCFE6FF050EBFEF21F018DF8C0EEF6E2A
:1045400027DF840EEF6E120031DFBF0EE926000E6A
:1045500012002CDFC30EE926000E12000BDF11EF54
:1045600022F0E66E3CEC26F0146E050EE15E14506F
:10457000120013DFE6521200FE0BEA36E96EC30E9C
:10458000E926000E1200FE0BEA36E96EBF0EE926A0
:10459000000E1200E1EC18F0146E060EE15E1450ED
:1045A0001200EA6ADE0FE96E000E1200EA6ADC0F02
:1045B000E96E000E1200E7DEEF50800B1200E3DE22
:1045C000E850EF16120094DFEE52080EEF6E78EF0F
:1045D00022F0020EE926000EEA221200D4DEE85094
:0445E000EF121200C4
:0C45E400019E08D0019E09AE05D0086CB5
:1045F000091EE86A0922018E09C003F008C002F012
:10460000136A126A8E0E046E056A20EF24F0016AA6
:104610005CEC24F074EC24F001B604EF24F001A269
:1046200005D001B804EF24F00BEF24F001AA05D067
:1046300001B004EF24F00BEF24F001B002D001A888
:1046400002D017EF24F0056A0F500A24046EE86ABE
:1046500005227E0E045EE86A055A126A136A026A2F
:10466000036A0E500902F4CF03F0F3CF02F00D50AD
:104670000902F3501326F4500222000E03220E50BA
:104680000802F3501326F4500222000E03220C50AD
:104690000902F3501226F4501322000E02220322C4
:1046A0000D500802F3501226F4501322000E02227D
:1046B00003220E500702F3501226F4501322000E6C
:1046C000022203220C500802F4501226000E13227C
:1046D000022203220D500702F4501226000E13226C
:1046E0000222032220EF24F0006AE86A0EAE81EF76
:1046F00023F00B6C0C1E0D1E0E1E0C220D220E2222
:10470000001E09AE8CEF23F0066C071E081E091E62
:10471000072208220922001E18EC26F009BEA3EF8A
:1047200023F000AE000C066C071E081E091EE86A86
:10473000072208220922026C031E041E051E032202
:1047400004220522000C00BE93EF23F00188FF0C29
:1047500009C013F008C012F008500D02F4CF07F0A2
:10476000F3CF06F009500E02F4CF09F0F3CF08F0B2
:104770000D02F3500726F4500822E86A092212506D
:104780000E02F3500726F4500822E86A09220EAE02
:10479000CEEF23F01250085E1350095A13AE000CEE
:1047A0000D50085E0E50095A000C016A5CEC24F0B2
:1047B00001B6DFEF23F001A20ED001B405D07F0EC9
:1047C000096EFF0E086E1FD0800E096E086A1BD09E
:1047D000096A086A18D001B0FBD78F0E0A60EDD7BE
:1047E0007E0E0A64F5D78E0E0A5C05E0D890093279
:1047F00008320A2AF8D701A406D0086C091EE86A14
:10480000092209AEE5D712007F0E0A6EFF0E096E6F
:10481000086E076E12007F0E01BEFF0E0A6E02D0F8
:104820007F0E0A6E800E096E086A076AF3D701AE22
:1048300004D0800E0A6E096AF7D70A6A096AF4D7AB
:104840000350021013101210F8E005BEF0D703BE9B
:104850000CD004500510EBE0D89012361336023617
:1048600003360406D8A00506F2D70550D4E1042883
:10487000D2E012AE11D07F0E121402E113A00CD0C0
:10488000132AE86A0222032207E3D88003320232A5
:104890001332042A0428BFE00450C9E013C007F013
:1048A00002C008F00334096E04300A6E09320A9E11
:1048B00001BE0A8E0AEF24F009360A3602E30184AB
:1048C000017E06E101800A6A096A086A076A120025
:1048D0000A2803E0D88009321200D890093202E198
:1048E00001821200018612000E360F3602E3018C9F
:1048F000017E06E101880F6A0E6A0D6A0C6A1200D9
:104900000F2803E0D8800E321200D8900E32EAE170
:04491000018A120006
:0C491400040120511F0B010801E01200FB
:10492000245101E01200060E215D1EE12351230AED
:104930001BE0010A0CE0030A17E10001B90514E1CC
:104940000001080EC96F4A0ECA6F090E09D0000196
:10495000B9050AE10001650EC96F4A0ECA6F2F0E34
:10496000CC6FCD6BC00ECB6F04012051600BE842C1
:10497000E842E842E842E842010801E01200215121
:104980000B0A2AE0080A1DE0090A15E0080A09E0F6
:104990000B0A05E0080A01E012009BEF19F0B1EFE5
:1049A00019F00001400EC96F040ECA6F010ECC6FE2
:1049B000CD6BC10E0FD00001800ECB6F23C440F42D
:1049C00012000001410EC96F040ECA6F010ECC6FB8
:1049D000CD6B810ECB6F12000001800ECB6F22C415
:0449E00041F412008C
:0C49E4001201000200000008D80412F8C4
:1049F00001000102000109022900010100C0320981
:104A00000400000203000000092111010001222F0F
:104A10000007058103400001070501034000010470
:104A20000309042A034D006900630072006F0063EC
:104A30000068006900700020005400650063006891
:104A4000006E006F006C006F00670079001803476C
:104A50000065006E00650072006900630020004878
:104A6000004900440006A0FF0901A1010903150047
:104A700026FF007508950481020904150026FF0031
:104A80007508950491020905150026FF0075089523
:0C4A900004B102C0F6491F4A234A4D4AF7
:044A9C001E0EF66E86
:104AA000100EF76E000EF86E04010900F5503B6F12
:104AB0000900F5503C6F03E13B6701D03DD0090090
:104AC000F550366F0900F550376F0900F550386F13
:104AD00009000900F550E96E0900F550EA6E090079
:104AE00009000900F550396F0900F5503A6F0900C7
:104AF0000900F6CF3DF4F7CF3EF4F8CF3FF436C4CB
:104B0000F6FF37C4F7FF38C4F8FF0401395302E158
:104B10003A5307E00900F550EE6E3907F8E23A071C
:104B2000F9D73DC4F6FF3EC4F7FF3FC4F8FF0401C8
:0A4B30003B07000E3C5BBFD71200EC
:064B3A00FF0EE366A3EF8D
:104B400025F0BFEF25F0FE0EE366A9EF25F0ABEFF1
:104B500025F0FF0EE32AFE0EE3060CE0E3060AE072
:104B6000E30608E000000000000000000000FE0E68
:104B7000E306F9E1FF0EE306F6E1CFEF25F0FE0EC6
:104B8000E3060DE0E3060BE0E30609E000000000A9
:104B90000000000000000000FE0EE306F9E1120034
:104BA000000EF36E00EE00F0080E01D81200EA606D
:104BB00002D0EE6AFCD7F350E9601200EE6AFCD72F
:104BC00006500B02F3CF02F0F4CF03F00C02F350C7
:104BD0000326000EF420046E06500D02F350042646
:104BE000000EF420056E06500E02F3500526075005
:104BF0000B02F3500326F4500422000E0522075046
:104C00000C02F3500426F450052207500D02F35015
:104C1000052608500B02F3500426F45005220850D4
:104C20000C02F350052609500B02F3500526120022
:104C3000056A046A036A026A200EE76ED890063697
:104C400007360836093602360336043605360B5069
:104C5000025C0C5003580D5004580E50055809E3DF
:104C60000B50025E0C50035A0D50045A0E50055A58
:084C7000062AE72EE4D712002A
:084C7800FE0EE3CFE9FFFF0E81
:104C8000E3CFEAFFE9CFF3FFEACFF4FFFB0EE350F7
:104C900003E1FC0EE35009E0FB0EE30602E2FC0E2A
:0C4CA000E306FD0EE350EE6EF1D71200AB
:044CAC00FF0EE350C4
:104CB0001D6EEF0E01D0F30EE76EE72E5DEF26F0CE
:104CC0000C0E1C6EE76AE72E63EF26F01C2E62EFD7
:0A4CD00026F01D2E5BEF26F0120007
:064CDA00056A046A100ED9
:104CE000E76ED89008360936043605360D50045C58
:104CF0000E50055805E30D50045E0E50055A082A63
:064D0000E72EF0D71200BF
:0A4D0600FF0EE3501D6E480E01D0B1
:104D10004C0EE76EE72EFED7E76AE72EFED71D2E74
:064D2000F7D700001200AD
:0A4D260013EE00F023EE00F0F86A2F
:104D3000019C4EEC25F003EC08F0DFEC0AF0FBD709
:024D400012005F
:0E4D4200FF0EE3501D6E1B0E00D001D0200EA0
:0E4D5000E76EE72EFED71D2EFAD700D0120018
:024D5E00010052
:104D60000000000000000000000000000000000043
:104D70000000000028000100010000000000000009
:104D80000000000000000000000000000000000023
:104D90000000000000000000000000000000000013
:104DA0000000000000000000000000000000000003
:064DB0000100000000728A
:020000040030CA
:0100000028D7
:010001000EF0
:010002003FBE
:010003001EDE
:010005008179
:010006008178
:010008000FE8
:01000900C036
:01000A000FE6
:01000B00E014
:01000C000FE4
:01000D0040B2
:00000001FF
